:020000000F28C7
:080008000B110900F6000030A5
:100010008A000F30760703188A0A76088207203094
:1000200083120313BB000430BC000230BD00D101B9
:1000300083120313D2010930D3000130D4000230FF
:10004000D5000130D6000230D7000830D80001308A
:10005000D90004308600F03083168500F230860027
:10006000403081008B01F0260730831203139F007C
:10007000193083169900243098009030831298002C
:100080008C01B7010130B600B901B8013030CC00A5
:100090006627B7010230B600B901B8014030CC0084
:1000A0006627FA30B400A327FA30B400A3272D271F
:1000B00083120313B7010230B600B901B801CC01B5
:1000C000662703240324831203130608F000F00CB0
:1000D000F00CF00C700C0F39F0007008063C031D9A
:1000E0007B2883120313A001A101A201A3018F3079
:1000F000A400E823D0297008073C031DFF28013025
:10010000831203135602031DB52805305202013035
:1001100003180301F1005208073C013003180301E2
:100120007104003C0319AE285208093C0130031940
:100130000301F10052080B3C013003190301710562
:10014000003C0319AE285208A000A101A201A3019E
:100150000730A400E82383120313CE00D20A0D3027
:100160005202031DD029D201D02902308312031379
:100170005602031DE52801305902031DC228023032
:10018000D900FE2802305902031DC9280330D900C6
:10019000E42803305902031DD0280430D900E42894
:1001A00004305902031DD7280530D900E428053052
:1001B0005902031DDE280630D900E4280630590212
:1001C000031DE4280130D900FE28033083120313F5
:1001D0005602031DFE28A001A101A201A301580897
:1001E000A400E82383120313CE0008305802031D35
:1001F000FC288830D800FE280830D800D0297008A4
:100200000B3C031D42290130831203135602031DC8
:100210001C290F305402031D0F290130D40054084B
:10022000BF007124013083120313A400E82383125A
:100230000313CE00D40AD02902305602031D2B2905
:10024000C4015908C50043250130A400E8238312E6
:100250000313CE00412903305602031D4129A0019A
:10026000A101A201A3015708A400E82383120313EC
:10027000CE00CE08031D3F298230D700412902302D
:10028000D700D02970080D3C031D87290130831247
:1002900003135602031D5729A001A101A201A301C6
:1002A0008130A400E82383120313CE00D02902304A
:1002B0005602031D67290130C4005908C5004325B3
:1002C0000130A400E82383120313CE0086290330F3
:1002D0005602031D86295308A000A101A201A30113
:1002E0000930A400E82383120313CE00093053021F
:1002F000031D7D294930D300862949305302031D4F
:1003000084298930D30086290930D300D029700888
:100310000E3C031DD0290430831203135502031D24
:1003200093290130D5003230B400A3275508F100DD
:100330007108013C031DA82983120313B701023081
:10034000B600B901B801CC0166270130D600CB292F
:100350007108023C031DB92983120313B70102304F
:10036000B600B901B8011030CC0066270230D600C3
:10037000CB297108033C031DCB2983120313B7015A
:100380000230B600B901B8012030CC006627033036
:10039000D600CB29CB2983120313D50AD029D02923
:1003A00083120313CD01C127553083120313CD00EF
:1003B000C12783120313CD01C12783120313CD017B
:1003C000C127BB3083120313CD00C127D027FE0005
:1003D000D027FF007E080139031DF7290130831261
:1003E0000313C100C2014130C3003525FF2901308C
:1003F00083120313C100C2014230C30035257E08B9
:100400004039003C03190C2A013083120313C10048
:10041000C2014D30C30035257E082039003C031948
:10042000192A013083120313C100C2014830C300EE
:1004300035250324F0013030F1002508F200F20CDC
:10044000F20CF20C720C0F3971070318F00AAA00B3
:10045000303C031D2D2A2030AA00F0013030F1007D
:100460002508F200720EF039F039F200F20CF20CAD
:10047000F20C720C0F3971070318F00AAB002A084E
:10048000203C0130031D0301F0002B08303C0130FB
:10049000031D03017005003C0319502A2030AB00F6
:1004A000F0013030F1002608F200F20CF20CF20CF0
:1004B000720C0F3971070318F00AAC002E30AD0032
:1004C000F0013030F1002608F200720EF039F039F8
:1004D000F200F20CF20CF20C720C0F3971070318D7
:1004E000F00AAE00F0013030F1002708F200F20C03
:1004F000F20CF20C720C0F3971070318F00AAF00FE
:10050000F0013030F1002708F200720EF039F039B6
:10051000F200F20CF20CF20C720C0F397107031896
:10052000F00AB0002E30B100F0013030F1002808A0
:10053000F200F20CF20CF20C720C0F397107031876
:10054000F00AB200F0013030F1002808F200720E1B
:10055000F039F039F200F20CF20CF20C720C0F3997
:1005600071070318F00AB3005108093C031CCD2A97
:100570000130C100F001023051070318F00AC20037
:1005800051082A3E84008313000883120313C3001A
:10059000352583120313D10AB42AD1010130CD00CD
:1005A000C127B63083120313CD00C1278312031372
:1005B000CD01C12783120313CD01C127BB308312A4
:1005C0000313CD00C127D027FE00D027FF007E08EF
:1005D000643C031DF52A013083120313C1000C3063
:1005E000C2002D30C30035250C2B7E08A43C031D12
:1005F000032B013083120313C1000C30C2002B30D7
:10060000C30035250C2B013083120313C1000C30BD
:10061000C2002030C300352583120313CD01C1274A
:10062000793083120313CD00C12783120313CD0148
:10063000C12783120313CD01C127BB3083120313DB
:10064000CD00C127D027FE00D027FF007E08003C48
:10065000031D2F2B343083120313D000452B7E084B
:10066000013C031D382B333083120313D000452B7C
:100670007E08023C031D3F2B3230D000452B7E0804
:10068000033C031D452B3130D0000230C100043043
:10069000C2005008C3003525831203132908BE0089
:1006A0002D24A001A101A201A301F730A400E82399
:1006B00083120313CE008039031D652B0230C10065
:1006C000C2015030C3003525822B02308312031340
:1006D000C100C2017330C300352583120313A0018A
:1006E000A101A201A301E730A400E82383120313B0
:1006F000CE008039031D822B0230C100C20153306D
:10070000C3003525831203134E08F000700EF03934
:10071000F039F000F00CF00CF00C700C0F39CF0039
:1007200001304F02031CC92B01304F020130031C62
:100730000301F0004F08093C0130031C0301700560
:10074000003C0319B72B0230C1000130C200F00198
:1007500030304F070318F00AC300352502308312EA
:100760000313C100C2002030C3003525DA2B02304C
:1007700083120313C1000130C2003930C300352594
:10078000023083120313C100C2002B30C300352591
:10079000DA2B023083120313C1000130C200203073
:1007A000C3003525023083120313C100C20020307C
:1007B000C3003525023083120313C1000630C20086
:1007C000F001303059070318F00AC30035256328BB
:1007D000831203132008CD00C127831203132108BD
:1007E000CD00C127831203132208CD00C127831235
:1007F00003132308CD00C127831203132408CD005F
:10080000C127D027080083120313CD01C12783120B
:100810000313CD01C12783120313CD01C127831216
:100820000313CD01C127033083120313CD00C12769
:10083000D02783120313A500D02783120313A60029
:10084000D02783120313A700D02783120313A80015
:10085000D02783120313A900080083120313DA01BF
:10086000DB01BE0803193E2C3E08F7000330F800F8
:10087000EC27F000780883120313BE005B08003CED
:100880000030031C4B2C0130031D4B2C5A08023C3A
:100890000130031C0301003C0319702C0130C1001E
:1008A0000030F0005B08F0070D305A070318F00A1B
:1008B000C200F00158303E070318F00A5A07F10051
:1008C0000318F00A5B08F0077108C0002D25831299
:1008D000C300352583120313DA0A0319DB0A3E2C01
:1008E0000800831203133F08F1007108013C031D47
:1008F000812C433083120313A000A101A201A301A4
:100900002C2D7108023C031D8E2C1430831203130E
:10091000A0005030A100A201A3012C2D7108033CBE
:10092000031D9B2C113083120313A0008030A10003
:10093000A201A3012C2D7108043C031DA82C083032
:1009400083120313A0008030A100A201A3012C2D6B
:100950007108053C031DB62C053083120313A0005B
:100960000130A1005030A200A3012C2D7108063CDB
:10097000031DC32C023083120313A0008430A10096
:10098000A201A3012C2D7108073C031DD02C0230BD
:1009900083120313A0004230A100A201A3012C2D59
:1009A0007108083C031DDD2C023083120313A000E4
:1009B0001430A100A201A3012C2D7108093C031DD4
:1009C000EA2C013083120313A0008230A100A2019F
:1009D000A3012C2D71080A3C031DF72C0130831252
:1009E0000313A0004230A100A201A3012C2D710825
:1009F0000B3C031D042D013083120313A000A10141
:100A00005030A200A3012C2D71080C3C031D112DA8
:100A100083120313A0017030A1005030A200A30183
:100A20002C2D71080D3C031D1E2D83120313A001F4
:100A30003630A1004030A200A3012C2D71080E3CDD
:100A4000031D2C2D83120313A0011830A100403088
:100A5000A200A3012C2D2C2D0800831203134008A3
:100A600083169B001C141A08080083120313410804
:100A7000CA004208CB003927831203130614430827
:100A8000C90016270800303083120313DC00393008
:100A9000DD004408003C0319522D5D08DA005C08B3
:100AA000DB00562D5C08DA005D08DB004508063CDB
:100AB000031C832E33085A020130031D0301F10089
:100AC000023045020130031C0301F2004508063CD8
:100AD0000130031C030172057104003C0319782ED8
:100AE00001304502031D762D5B08B30032085A021F
:100AF0000130031D0301F100033045020130031CE6
:100B00000301F2004508063C0130031C0301720595
:100B10007104003C03196D2E4508013C0130031D92
:100B20000301F1004508023C0130031D030171047B
:100B3000003C03199D2D5B08B20030085A020130B9
:100B4000031D0301F100043045020130031C0301C1
:100B5000F2004508063C0130031C030172057104D4
:100B6000003C0319622E013045020130031C0301D1
:100B7000F1004508033C0130031C03017105003CF2
:100B80000319C42D5B08B0002F085A020130031D61
:100B90000301F100053045020130031C0301F2009E
:100BA0004508063C0130031C030172057104003C3A
:100BB0000319572E013045020130031C0301F100D7
:100BC0004508043C0130031C03017105003C031976
:100BD000EB2D5B08AF002E085A020130031D030104
:100BE000F1004508063C0130031D03017104003C7F
:100BF00003194C2E013045020130031C0301F100A2
:100C00004508053C0130031C03017105003C031934
:100C10000B2E5B08AE002C085A02031D412E01303A
:100C200045020130031C0301F1004508063C013078
:100C3000031C03017105003C0319202E5B08AC0066
:100C40002B085A02031D362E5B08AB002A085A02F5
:100C5000031D2D2E5B08AA00832E2A08C600440817
:100C6000C7000130C800DE26AA00832E83120313BA
:100C70002B08C6004408C7000130C800DE26AB00C0
:100C8000832E831203132C08C6004408C7000130CA
:100C9000C800DE26AC00832E831203132E08C60084
:100CA0004408C7000130C800DE26AE00832E831240
:100CB00003132F08C6004408C7000130C800DE2611
:100CC000AF00832E831203133008C6004408C70008
:100CD0000130C800DE26B000832E831203133208D1
:100CE000C6004408C7000130C800DE26B200832ECB
:100CF000831203133308C6004408C7000130C8003C
:100D0000DE26B300832EF101831203132A08F200BA
:100D1000720EF039F039F2002B08F300730EF0393F
:100D2000F039F300F30CF30CF30C730C0F3972076A
:100D30000318F10AA000F1012C08F200720EF0393C
:100D4000F039F2002E08F300730EF039F039F30099
:100D5000F30CF30CF30C730C0F3972070318F10A40
:100D6000A100F1012F08F200720EF039F039F20003
:100D70003008F300730EF039F039F300F30CF30C84
:100D8000F30C730C0F3972070318F10AA200F1017A
:100D90003208F200720EF039F039F2003308F30035
:100DA000730EF039F039F300F30CF30CF30C730C01
:100DB0000F3972070318F10AA30008008312031306
:100DC0004708003C0319EB2EF101460848070318B9
:100DD000F10AC600EE2E48084602C6004608080082
:100DE00083120313861106100530B400A3270330C5
:100DF000850028270530B400A32702308500282766
:100E00000530B400A3272830C90016270830831204
:100E10000313C90016270C3083120313C9001627C9
:100E2000063083120313C900162708008312031328
:100E30004908F300F30CF30CF30C730C0F39850025
:100E400028274908850028272830BA00B427080039
:100E500083120313861586110800831203130610EC
:100E60000130C9001627023083120313B400A327F0
:100E700008008312031306104A08F2007208013CAE
:100E8000031D4C2FF3018030831203134B0703180B
:100E9000F30AC9001627602F7208023C031D602F59
:100EA000F3014030831203134B070318F30AF400D5
:100EB00073080038F30074088038C9001627602FC3
:100EC000023083120313B400A32708008312031314
:100ED000DA01DB015B08003C0030031C772F013096
:100EE000031D772F5A080F3C0130031C0301003CFF
:100EF0000319A22F3708F2003608CA003908F20099
:100F00005B08F20738085A070318F20ACB003927A2
:100F10008312031306140030F2005B08F2074C083A
:100F20005A070318F20AC0002D25013CF20072098D
:100F3000013E8312C900162783120313DA0A03192C
:100F4000DB0A6A2F08008E3083120313B5000000FD
:100F500000000000000000000000B50BA92F0000F9
:100F6000B40BA32F0000080083120313BA0CBA0CB1
:100F70003F30BA050330BA020000BA0BBC2F0000A4
:100F80000800831203134D0899008316831203137C
:100F900001080319CE2F83161808C62F83120800E4
:100FA000831203130C083B05FF39003C0319D02FB3
:100FB00018083C05FF39F10018083D05FF39710498
:100FC000003C0319E82F1812000018161A08DE005A
:100FD0001A080800D02F08000930F9007708F70137
:100FE0000310F70CF80C0318F707F90BF12F77082B
:020FF0000800F7
:02400E00503F21
:1042000021002100210021002100210021002100A6
:104210005700670021004300650021004E00650043
:104220002100210021002100210021002100210086
:1042300056007100210045007800210054007500EF
:104240002100210021002100210021002100210066
:1042500053007100210054007100210051005500ED
:10426000470055002E00390032003800210053006D
:1042700066006E007000750066004E0062006F0000
:104280004A00580033004D004700450021007300EC
:1042900032002F00320021003300310031003500A0
:1042B0004C005300420055005300420020004300D0
:1042C0005700430057005200200041004D000000FD
:1042D00000000000570046004D00000000000000F4
:1042E000200046004D00000000000000440049008E
:1042F000470000000000000050004B005400000088
:00000001FF
